:020000040000FA
:040000001DEF00F000
:0200080014D012
:08001800D8CF81F0E8CF80F0A1
:10002000E0CF82F082C0E0FF80C0E8FF81C0D8FF4F
:100030001000F2B486ED04F011000F01060EC16E3F
:100040000F01386B396B3A6B3B6B3C6B210E926E38
:10005000C00E936E030E946E000E956E968096926F
:100060009694720ED36E0F0100EE00F000EC03F0D8
:1000700080EC04F08B848B8682A23CEF00F08B84B2
:10008000C0EC03F00E828B9606EC03F006EC03F056
:1000900006EC03F006EC03F082A251EF00F068EFEB
:1000A00000F073EC03F006EC03F006EC03F006EC52
:1000B00003F006EC03F082A060EF00F068EF00F0C0
:1000C0008B8645EC04F017803FEF00F066EF00F000
:1000D0000A6A0C6A0B6A0D6A076A086A0E920E9029
:1000E0000970097206EC03F068EF00F076EF00F09B
:100600000400EE6AEAA400EF03F01200FF0E106E81
:10061000FF0E116E80BAFF00112E0AEF03F0102EAC
:1006200008EF03F01200126EFF0E136EFF0E146E31
:1006300080BAFF00142E18EF03F0132E16EF03F00C
:10064000122E14EF03F01200070E166E010E076E45
:10065000040E13EC03F00746040E13EC03F0162E01
:100660002BEF03F0076A070E166E010E086E040EDC
:1006700013EC03F00846040E13EC03F0162E3AEFC9
:1006800003F0086A24EF03F0070E166E010E076EE2
:10069000040E13EC03F00746040E13EC03F0162EC1
:1006A0004BEF03F0076A030E166E010E086E040E80
:1006B00013EC03F00846040E13EC03F0162E5AEF69
:1006C00003F0086A1200070E166E800E0C6E040E00
:1006D00013EC03F00C42040E13EC03F0162E6AEF39
:1006E00003F00C6A12000A0E166E0888040E13EC52
:1006F00003F082A079EF03F00898088A040E13EC47
:1007000003F082A081EF03F0089A088C040E13EC2A
:1007100003F082A089EF03F0089C088E8B94040EEE
:1007200013EC03F08B84089E0E80040E13EC03F090
:100730000E90162E75EF03F0120008880A0E13ECC7
:1007400003F00898088A0A0E13EC03F0089A088848
:10075000088C0A0E13EC03F00A0E166E089C08981B
:10076000088A088E0A0E13EC03F0089A089E08887F
:10077000088C0A0E13EC03F0162EAEEF03F01200F5
:10078000DF0E0A6E0B8AFF0E0C6E0A0E166E17B085
:10079000DBEF03F006EC03F082B2DBEF03F08B86B5
:1007A0000980099206EC03F00990098206EC03F037
:1007B000162ED0EF03F007800C9E0D8E0B9A0A8A3E
:1007C0000A980B88080E13EC03F082A2E5EF03F001
:1007D00007820D9E0C8E0C9C0D8C0B980A880A9635
:1007E0000B86080E13EC03F082A2F4EF03F00784EB
:1007F0000D9C0C8C0C9A0D8A0B960A860A940B841D
:10080000080E13EC03F082A203EF04F007860D9AA2
:100810000C8A0C980D880B940A840A920B82080E9D
:1008200013EC03F082A212EF04F007880D980C88F5
:100830000C960D860B920A820A900B80080E13EC20
:1008400003F082A221EF04F0078A0D960C860C9427
:100850000D840B900A80080E13EC03F082A22EEF99
:1008600004F0078C0D940C840C920D82080E13EC8E
:1008700003F082A239EF04F0078E0D920C820C90E7
:100880000D8082A241EF04F0120008800D900C80D0
:100890000A9E0B8E080E13EC03F008820B9E0A8E44
:1008A0000A9C0B8C080E13EC03F008840B9C0A8C3A
:0C08B0000A9A0B8A080E13EC03F01200E9
:10090000C30ED56EF28CF28AF28E1200F29480BA87
:10091000FF000FB29BEF04F00FB4B6EF04F00FB678
:10092000D9EF04F00FB8FCEF04F00FBA1FEF05F099
:100930000FBC3EEF05F08A6A8C6A8B988B9A8B9C71
:100940008B9E8998899289948D928D940AB88A8019
:100950000BB88A860ABE8C8E0BBE8C880CB68B8E2A
:100960000DB68B8C89860F6A0F8412008A6A8C6A96
:100970008B988B9A8B9C8B9E8996899289948D9269
:100980008D940AB08C800BB08A8A0ABA8A800BBA1E
:100990008A860ABC8C8E0BBC8C880CB88B8E0DB8EA
:1009A0008B8C0EB08B8A0EB28B8889880F6A0F866B
:1009B00012008A6A8C6A8B988B9A8B9C8B9E899882
:1009C000899689948D928D940AB28C800BB28A8A12
:1009D0000AB48A800BB48A860CB28C8E0DB28C88D5
:1009E0000CB48B8E0DB48B8C0CBE8B8A0DBE8B8899
:1009F00089820F6A0F8812008A6A8C6A8B988B9A98
:100A00008B9C8B9E8998899289968D928D9409B042
:100A10008A8A09B28C800AB68A800BB68A860CB0A4
:100A20008C8E0DB08C880CBA8B8E0DBA8B8C0CBC56
:100A30008B8A0DBC8B8889840F6A0F8A12008A6AA0
:100A40008C6A8B988B9A8B9C8B9E899889928994BF
:100A500089968D9407B28A8807B48A8407BA8A82F5
:100A600007BE8C8C08B28C8A08B48C8208B88C843F
:100A700008BE8C868D820F6A0F8C12008A6A8C6A7F
:100A80008B988B9A8B9C8B9E8998899289948D9256
:100A9000899607B08A8807B68A8407B88A8207BC15
:100AA0008C8C08B08C8A08B68C8208BA8C8408BCFE
:0C0AB0008C868D840F6A0F8212001200E9
:020000040030CA
:0300010028183C80
:02000500BD81BB
:060008000FC00FE00F40E5
:00000001FF
